:020000020000FC
:1000000030C2189518951895189518951895189543
:10001000189518951895DFC1189518951895189585
:10002000189518951895189518950C006000DC0423
:1000300040E050E060E070E0002391F0102F4F5F4F
:100040005F4F6F4F7F4F483002E5500700E0600779
:100050007007ACF340E050E060E070E01A9579F78B
:1000600000E010E020E030E00895392F482F5D9B3C
:10007000FECF00E10CB95D9BFECF0CB9E0E6F0E0ED
:1000800003815D9BFECF0CB95D9BFECF00E10CB9F7
:100090000081118116950795169507955D9BFECFFA
:1000A0000CB980E090E000811181012BA9F0228140
:1000B00085BB092F0F70022B08BB00ED02BB02BBF2
:1000C00009B35D9BFECF0CB900EF02BB0196008126
:1000D00011818017910760F300EF02BB842F932FEB
:1000E000089500EF02BBE0E608EFF0E0038300E0D4
:1000F00010E020E030E0548140E742BB42BB42BB0D
:1001000040EF42BB8299FECF40EA42BB69B340EF69
:1001100042BB651718F409EF03830AC00F5F1F4F36
:100120002F4F3F4F01301F0741E024073F0724F3C3
:1001300000E010E020E030E0558140E742BB42BBE8
:1001400042BB40EF42BB8299FECF40EA42BB69B35B
:1001500040EF42BB561720F40381026003830AC0BC
:100160000F5F1F4F2F4F3F4F01301F0741E0240704
:100170003F071CF300EF02BB089500EF02BBE0E66F
:1001800008EFF0E0038300E010E020E030E054816D
:1001900040E742BB42BB42BB40EF42BB8299FECF2D
:1001A00040EA42BB69B340EF42BB561718F409EF6F
:1001B00003830AC00F5F1F4F2F4F3F4F01301F07B0
:1001C00041E024073F0724F300E010E020E030E0A6
:1001D000558140E742BB42BB42BB40EF42BB8299E4
:1001E000FECF40EA42BB69B340EF42BB651720F443
:1001F0000381026003830AC00F5F1F4F2F4F3F4FE1
:1002000001301F0741E024073F071CF300EF02BB4A
:10021000089500E702BB02BB02BB10E000E0309192
:10022000610015BB4091620048BB20EF22BB22BB9E
:1002300022BB20EB22BB8299FECF20EA22BB20E723
:1002400022BB139515BB89F70395242F202B28BBC0
:10025000031759F748BB00EF02BB07CF40E050E05F
:1002600060E070E01124002389F0102F04C04F5F7C
:100270005F4F6F4F7F4F4017510561057105BCF30C
:1002800040E050E060E070E01A95A9F708954A92C6
:10029000BA93AA939A938A93402F00EF02BB80E00F
:1002A00090E0A091610085BB4090620048BA01E0F7
:1002B00010E0E4D0B02F00E702BB02BB02BB00EFAE
:1002C00002BB8299FECF00EA02BB00EF02BB0B2FFC
:1002D000C5DF839585BB79F79395042D092B08BB62
:1002E0009A1749F748BA00EF02BB02BB829BFECFC8
:1002F000BCDE89919991A991B99149900895402FB7
:10030000475000EF02BB0091620008BB00E702BB50
:1003100002BB02BB00EF02BB8299FECF00EA02BB28
:1003200009B35D9BFECF0CB901E010E0A7D080DEE1
:1003300000EF02BB829BFECF089500E00ABB0FE1F5
:1003400007BB00E108BB0FEF04BB00E005BB08EFF3
:1003500001BB00EF02BB00E000BD00E109B9599A02
:1003600008E90AB900E100BD789404E161DE00EF1C
:1003700002BB01C04EDF00EF02BB02BB00E702BBC5
:1003800002BB02BB00EF02BB8299FECF00EA02BBB8
:1003900002BB02BB00EF02BB02BB02BB829BFECFD3
:1003A00008EFE0E6F0E003830781013039F40581CE
:1003B0001481011710F095DE01C0DFDEE0E6F0E009
:1003C00016811123B9F2012F0A95183010F45FDF5E
:1003D000D2CF95DFD0CFFA93EA931A920A924A933A
:1003E0003A932A931A930A934FB7E0E6F0E0118507
:1003F000108722852187038502873CB133871F3F01
:1004000011F52E3F01F5132F083029F404E0109F59
:100410000082118218C0003111F4368314C00131FA
:1004200039F4332319F000E102830DC0F2830BC0CD
:10043000003211F4378307C0013211F4348303C052
:10044000023209F435834FBF0991199129913991ED
:10045000499109901990E991F991189500008895B2
:10046000FECF0BEA0DBF00E00EBFCCE8D0E00CD011
:10047000002309F019D061DFF1DFF0CF4A951AF0BF
:10048000000F111FFBCF089501E0089520E006D072
:10049000E9F70895259102D0E9F708952D930150C9
:1004A0001040202F212B08958AE290E0FC01059155
:1004B0001491FC013296A591B491FC0134962591DA
:1004C0003491422F432B19F0F901E4DF01C0DEDF44
:1004D000069610E08033910748F30895000310F862
:0804E000848604000000000006
:0400000300000000F9
:00000001FF
